:020000040000FA
:0400000004303A2866
:08000800A000030EA100831209
:1000100005191028831601178312B23081002B288E
:1000200083160113831203140B190310A80DA90DD5
:10003000AA0DAB0DAC0DAC16FF302C02031D2B2806
:10004000FA302B02031D2B2831152A08AF0029088E
:10005000AE002808AD008B100B11210E8300A00EFE
:04006000200E090065
:0C007400203084008001840A6030040207
:10008000031C3C281230B00086218316FF23900009
:10009000831283160C308505870183128501870141
:1000A000073099000030831691009F008312C830FA
:1000B00083168100831231309000003083168C004B
:1000C000831210308B00831600309B001C141A081A
:1000D0008312BC00831610309B001C141A08831274
:1000E000BD00E221831620309B001C141A088312E5
:1000F000C2000130C21BC200C2080319C200810144
:100100008E018F010B118B100B108C018B17962019
:1001100031199920B30B9428031085190314B90DD4
:10012000F030390203190921E321872864003210D5
:10013000080031110130B7008B13203037078316C8
:100140009B001C141A088312A40010303707831672
:100150009B001C141A088312A300A6000230A606F6
:100160000030370783169B001C141A088312A20064
:10017000A7000130A7068B17321CC42822090339B7
:10018000A200A309A409A50924082F02031D03291D
:1001900023082E02031DE52822082D02031D032932
:1001A00001303702031DD7283D143E148721023049
:1001B0003702031DDE28BD143E149321033037029D
:1001C000031DE5283D153E149F2126082E02031D20
:1001D000032927082D02031D032901303702031DBF
:1001E000F4283D103E14B02102303702031DFB28D5
:1001F000BD103E14B12103303702031D02293D1109
:100200003E14B2210329B70A04303702031808004C
:100210009C280130B600B300B400B500B7008501DA
:100220008701B113D1219620B30B3629031085190C
:100230000314B90DF030390203195D29B41F85018B
:10024000B41F8701B40B3629B50B36290230B5002F
:10025000013037020319B821023037020319BD21DA
:10026000033037020319C721FA30B400311D1329B6
:100270003111321C40292D090339AD00AE09AF09F7
:100280002F1C13298E018F010C1C13290C102E1EFC
:1002900013298B1320303707BB002F08BA007321B6
:1002A00010303707BB002E08BA0073210030370723
:1002B000BB002D08BA0073218B17D421850187015B
:1002C000B70AB60104303702031C1329C001080025
:1002D000E22108003E1C08003E101030BB003D0823
:1002E000BA00732108008B133A0883161C159A0074
:1002F0003B089B0055309D00AA309D009C14640073
:100300009C187F291C1183128B1708000800851682
:10031000051285100510C001C0148E018F010C104C
:100320004208C10008008516051285100510C0019D
:1003300040158E018F010C104208C1000800851283
:10034000051285140510C001C0158E018F010C1017
:100350004208C10008000800080008000800080062
:10036000080008000800080008000800080008004D
:10037000380903398500B8000800C00A3809333944
:10038000B800C01C0339C01830398500080038098E
:1003900030398500B800080008000800080008008F
:1003A0000800B801B8140800B80101303702031D75
:1003B000DB29B814381602303702031DE12900008A
:1003C000B816080008000C1C87280C10C10B8728E1
:1003D0004208C1008501C018051440198514C019D0
:1003E0000516C0018E018F010C104208C1000800E3
:084000000300030003000800A7
:02400E00CC01E3
:10420000010078007A007C007E007B0079007F004E
:104210007D007A0078007E007C00FF00FF00FF0038
:104220000000F200F600FA00FE00F200F600FA00CC
:10423000FE00F200F600FA00FE00FF00FF00FF00A3
:10424000010005000500050005000900090009003E
:1042500009000D000D000D000D00FF00FF00FF0024
:10426000FF00FF00FF00FF00FF00FF00FF00FF0056
:10427000FF00FF00FF00FF00FF00FF00FF00FF0046
:10428000FF00FF00FF00FF00FF00FF00FF00FF0036
:10429000FF00FF00FF00FF00FF00FF00FF00FF0026
:1042A000FF00FF00FF00FF00FF00FF00FF00FF0016
:1042B000FF00FF00FF00FF00FF00FF00FF00FF0006
:1042C000FF00FF00FF00FF00FF00FF00FF00FF00F6
:1042D000FF00FF00FF00FF00FF00FF00FF00FF00E6
:1042E000FF00FF00FF00FF00FF00FF00FF00FF00D6
:1042F000FF00FF00FF00FF00FF00FF00FF00DD00E8
:00000001FF
